:10000000E5C0FFC0DFC2FDC0FCC0FBC0FAC0F9C044
:100010006BC3F7C0F6C0F5C0DDC3F3C0F2C018CDA6
:10002000F9CC25CD2FCD39CD46CD63CD00000000D4
:10003000A60EF9154C1DF22B3E498A6601020304F7
:10004000050607030303030414E6FF0000005AFF3C
:10005000FFFF000046FF1EFF000050FF1EFF0000D4
:1000600019FFFFFFFF00256E183F96FFFFFF0000FE
:10007000000000468CFF146EFFFFFF0000000738F1
:1000800089FF1E78FFFF0000000050FF1EFFFF00E9
:10009000000050FF78FF000046FFFF0000FF00FF58
:1000A0000000000000000000000000000000000050
:1000B0000000000000000000000000000000000040
:1000C0000000000000000000000000000000000030
:1000D0000000000000000000000000000000000020
:1000E00000020304050708090B0C0E0F1112141669
:1000F00017191B1D1E20222426282A2C2F313335A8
:10010000383A3C3F424447494C4F5255575A5D603C
:1001100064676A6D7174777B7E8286898D9195990B
:100120009DA1A5A9ADB2B6BABFC4C8CDD2D6DBE0F9
:10013000E5EAEFF4FAFF03030304040405050606E9
:100140000708090A0B0C0D0E0F11121416181A1CB1
:100150001E212326292C2F33363A3E42464A4F533E
:10016000585D63686E747A80878E959CA4ACB4BC2D
:10017000C4CDD6DFE9F3FDFFFFFFFFFFFFFFFFFF69
:10018000FFFFFFFFFFFFFFFFFFFFFFFFFFFFFFFF7F
:10019000FFFFFFFFFFFFFFFFFFFFFFFFFFFFFFFF6F
:1001A000FFFFFFFFFFFFFFFFFFFFFFFFFFFFFFFF5F
:1001B000FFFFFFFFFFFFFFFFFFFFFFFFFFFFFFFF4F
:1001C000FFFFFFFFFFFFFFFFFFFFFF0011241FBE28
:1001D000CFE5D2E0DEBFCDBF10E0A0E6B0E0E0EDBD
:1001E000FBE102C005900D92AA39B107D9F720E0D2
:1001F000AAE9B0E001C01D92A13FB207E1F767D7BD
:10020000E5CCFECE20ED37E0019720F0F9013197E3
:10021000F1F7FACF08959091E900992349F08823E6
:1002200021F083E187BBC49A089583E087BBC4981B
:100230000895815090E0FC01E056FF4F2491FC01AD
:10024000EA5CFE4F849189BD28BD8091E50088233A
:1002500011F080E0E0CF0895CF93DF93E091EA00C2
:10026000F0E0E45CFF4F84918093DF001092CB00BC
:100270001092D5009091EF00992341F09091EE00FB
:100280009093D6001092CC0092E001C091E020E063
:1002900030E0482F50E0692F70E0241735072CF527
:1002A000A091EA00B0E0AA0FBB1FAC59BF4FED917F
:1002B000FC91E20FF31FE491E901C60FD71FDE01A5
:1002C000AB52BF4FEC93A091EA00B0E0AA0FBB1F66
:1002D000A458BF4FED91FC91E20FF31FE491C55379
:1002E000DF4FE8832F5F3F4FD8CF890F8093DF0028
:1002F000DF91CF910895811108C019BC18BC80917D
:10030000E500882319F081E086CF93CF089581E03E
:100310008093CA0093E09093EE0025E02093C800FC
:1003200022E02093E3009093EA008093EF00109284
:10033000C9001092ED008093EC001092E0008093D1
:10034000E9000895CF93DF931F92CDB7DEB79FEFFB
:1003500098BD90E0698356DF18BC6981862F90E0D4
:100360000F90DF91CF914ECF8091CA008093B7005C
:100370001092CA001092F0008BE58093B90080E0E3
:100380004ACF8091B7008093CA001092C400809138
:10039000CA00882319F01092B90008958091B8001E
:1003A0008093B9000895EF92FF920F931F93CF931C
:1003B000DF93C82F8B017B01EE0CFF1CEE0CFF1CA2
:1003C000D8E2CC2371F081E026DFD9BD18BCC8018A
:1003D00019DF80E020DF19BC18BCC70113DFC15052
:1003E000F0CFDF91CF911F910F91FF90EF90089583
:1003F0001F93CF93DF93C82FD62F18E2CC2301F1A0
:100400008091B9008D131CC081E005DF8091E90067
:10041000882321F08091E000811102C019BD18BC31
:100420008AEF90E0EFDE80E0F6DE19BC18BC87E7CB
:1004300091E0E8DE8091B9008D1302C0C150DECF9B
:10044000DF91CF911F9108951F93CF93DF93D62F04
:100450006AE081DB192F6D2FCBDFC091B900CD137E
:1004600010C080E293E0CEDE6C2F812FC1DF80913F
:10047000B9008C1306C080ED97E0DF91CF911F91FA
:10048000C1CEDF91CF911F910895EF92FF920F930C
:100490001F93CF93863018F006E910E002C00AEFF0
:1004A00010E07801EE0CFF1CC82FCC23D1F019BC52
:1004B00018BCC801A7DE81E0AEDE8091CA008823A7
:1004C00021F08091E20017DF06C08091C700909173
:1004D000E10099BD88BDC70195DE80E09CDEC1507A
:1004E000E4CFCF911F910F91FF90EF900895EF927D
:1004F000FF920F931F93CF938C017C01F594E794A7
:10050000C62FCC2351F081E086DEC8017BDE80E07F
:1005100082DEC70177DEC150F4CFCF911F910F91DA
:10052000FF90EF900895CF93C82F68E270E082E0CB
:100530003ADF80EF90E066DE64E670E08C2F33DF18
:100540001092BA00CF91089586B383FB882780F973
:1005500091E098278091A200880F892B8093A200B8
:100560009091A100992311F08F7001C08170809348
:10057000A1008091A10090E008958091B9008031A0
:1005800020F48091B9008093B8008091B9008F5F0A
:100590008093B9009091DF00891710F01092B90094
:1005A00008958091B9008093B8008091B9008111BD
:1005B00003C08091DF0002C08091B9008150809318
:1005C000B900089518958EBB6DBB84E28CBB86E2A2
:1005D0008CBBE199FECF0895CF93DF932091B900B2
:1005E0008091EA009091CA00880F880F880F979534
:1005F00099279795692F682B622B6093EB002091C8
:10060000C9003091ED009091EE008091C800330F49
:10061000990F990F932B922B8295880F807E892BAF
:100620008093C6004091C5005091E9003091EC00E4
:100630009091E0008091EF007091E300550F330F2F
:10064000330F352B342B990F990F990F292F232B0B
:100650008295807F982F922B872F8295880F807E9E
:10066000892B8093E700C091A300D091A400CE0114
:1006700004968F7799279093A4008093A300A3DF1B
:100680008091A3006091C6008F5F9DDF8091A300E1
:100690006091E7008E5F97DFCEBB84E18CBB86E183
:1006A0008CBBE199FECF8C2F8F5F8EBB84E18CBB1E
:1006B00086E18CBBE199FECF8C2F8E5F8EBB84E1EF
:1006C0008CBB86E18CBBE199FECFCD5FCEBB84E1D4
:1006D0008CBB86E18CBBE199FECF8091A3006DE5D8
:1006E0008D5FDF91CF916FCF1F920F920FB60F9258
:1006F00011245F936F937F938F939F93AF93BF93D7
:1007000064B175B18091A800813021F5CB01969537
:100710008795945D2CDA6E5F7F4F8091AA008823C5
:10072000B9F08091AA0090E08617970728F480918D
:10073000AA008F5F8093AA008091AA0090E06817BA
:10074000790740F48091AA0081508093AA0002C0EA
:100750006093AA008091A8008330F9F4665171403B
:100760008091A9008823B9F08091A90090E08617B4
:10077000970728F48091A9008F5F8093A90080914A
:10078000A90090E06817790740F48091A900815092
:100790008093A90002C06093A9008091A8008F5F98
:1007A0008093A800843010F01092A8008091A800D7
:1007B000823010F48CE001C08FE887B9BF91AF910F
:1007C0009F918F917F916F915F910F900FBE0F90CE
:1007D0001F9018951F920F920FB60F9211242F930E
:1007E0003F934F935F936F937F938F939F93AF93B9
:1007F000BF93EF93FF938091E800882321F081500D
:100800008093E80053C48091A6009091A700892BA3
:1008100049F08091A6009091A70001979093A700BE
:100820008093A60091DE2091B5003091B600892B0F
:1008300009F4C0C1203D87E0380730F42F5F3F4FF7
:100840003093B6002093B5008091B5009091B6002A
:10085000823E24E0920771F41092C4001092E200EC
:100860001092B9001092C30081E08093BE001092F4
:10087000BD001CC43091BD002091AE003323B1F007
:100880001092BA00211112C48332910521F4809193
:10089000BD008F5F08C08634910509F007C481E070
:1008A0008093AE008FE08093BD0000C4211177C11A
:1008B0002091CA00222309F49DC0429708F49AC0EF
:1008C0008091BE00811196C08091BF00811192C0BD
:1008D0008091B900803508F08DC08091C3008130CF
:1008E00009F459C038F0823009F45DC0833009F44E
:1008F00064C080C08091C400811120C081E08093D9
:10090000C30087E18093E4008091EE0089BD18BCAC
:100910008091E500882311F080E07DDC8FEF8093EB
:10092000C4008093E2008091C000811104C08091D6
:10093000C4008093C0001092C1005CC08091C100CF
:100940009091C200882329F09093C3001092C100B7
:1009500004C085E0891B8093C3008091C400863960
:1009600021F493E09093C3000AC08091C4008F3FAC
:1009700051F482E08093C30081E08093C4008093AF
:10098000E20057DC37C08091C400813099F582E0E5
:100990008093C3002FC08091E40081508093E400D5
:1009A000811128C0E6CF8093C2008091C4008639AF
:1009B000B0F48091C4008F5F09C08093C200809121
:1009C000C400823060F08091C40081508093C400E4
:1009D0008093E2008091C4008093C00008C084E04E
:1009E0008093C30080E087DC87E090E00BDC80919F
:1009F000E20081DC8091CA0081112CC08091B50099
:100A00009091B600489731F58091BE00811122C0C7
:100A10008091B900803140F48091C900882311F0A1
:100A2000ACDD18C0BEDD16C08091B9008B3590F0EA
:100A3000E091F000EE2351F0E150E093F000F0E09F
:100A4000EC56FF4F80818093B90004C081E0809311
:100A5000BF0097DC8091B5009091B6008B34910572
:100A600009F06EC08091B400823009F58091B10028
:100A70009091B2000E97D8F48091CA00882329F093
:100A80008091BE00813009F05BC01092C4001092CA
:100A9000E2001092B9001092C3009091BE0081E074
:100AA000282F291B2093BE008093BF0049C080914E
:100AB000BE00811145C08091B400813099F420912D
:100AC000B1003091B2002E30310560F49091CA002F
:100AD000911136C090E59093B9008093BF0019BC86
:100AE00018BC2EC08091B9008B3510F04ADC28C0AC
:100AF0008091B900803531F41092B90019BC18BC4E
:100B000085E109C08091B900823569F41092B9007D
:100B100019BC18BC8EE08093BD001092BB0081E030
:100B20008093AE000DC08091CA00811109C08091F0
:100B3000E300882329F08091B900803509F014DCA6
:100B40008091BE0081112BC08091CA0081110FC01D
:100B50008091B5009091B600883C910541F4809158
:100B6000B400823021F08091B900803559F4809131
:100B7000CA008823A1F08091B5009091B600843F0F
:100B8000914069F41092B9001092C4001092C30011
:100B900019BC18BC81E08093BD001092BB0010927C
:100BA000A00010929F0088E391E0909361008093F1
:100BB000600072C21092AE008091BD008823A1F047
:100BC0002115310559F02831310528F48091BB00F9
:100BD0008F5F8093BB001092BA005AC28091BA0016
:100BE0008F5F8093BA0054C22115310509F426C1E4
:100BF0008091CA00882309F47BC01092C30022317F
:100C0000310508F069C08091B4008F5F8093B40013
:100C10008091B400813009F068C08091B900809360
:100C20009E008091B900803138F48091C4008639EB
:100C300019F48FEF80939E008091B900803541F0C8
:100C40008091B900813521F08091B900823549F455
:100C50001092B9001092C4001092E20081E08093DB
:100C6000BF008091BE00811140C08091BF00811102
:100C70003CC08091C40081111AC08091C0008111D4
:100C800003C081E08093C00081E08093C10092E0C6
:100C90009093C2009091C0009093C4009093E200A2
:100CA0009091E900992339F08093A50004C0109237
:100CB000C4001092E2008091E2008F3F59F48091CD
:100CC000EE0089BD18BC8091E500882371F080E0BA
:100CD000A2DA0BC010DB09C01092B4008091E900C9
:100CE000882319F081E08093A5001092BF00A1C075
:100CF0002831310508F081C08091B900803541F07C
:100D00008091B900813521F08091B900823561F47C
:100D10008091B90080939E001092B9008091B40038
:100D20008F5F8093B40085C08091B900811106C0A7
:100D30008091B400811102C081E007C08091B400AD
:100D4000882329F08091B4008F5F8093B400809154
:100D5000BE0081116EC08091ED00882379F08091F2
:100D6000B300882359F08091B900811107C08091A8
:100D7000B3008093B9001092B3005BC08091B900BA
:100D80008031F0F48091B900882391F08091B10016
:100D90009091B2008B34910558F08091B900809306
:100DA000B3008091B9008093B8001092B90041C09F
:100DB0008091C900882311F0F4DB3BC0DEDB39C031
:100DC0008091B1009091B2008B34910510F0D9DA86
:100DD00030C08091E3008130D1F3E091F000EF5F0B
:100DE000E093F00080916300E81788F7F0E0EC569C
:100DF000FF4F80818093B9001CC02B343105B8F4BB
:100E00008091B400813099F42091B1003091B2000A
:100E10002E30310560F49091B900911108C0909185
:100E2000E500891B8093E5008091E500F4D91092DC
:100E3000B4001092B2001092B1002AC18091B100AA
:100E40009091B20001969093B2008093B100892BEB
:100E500031F480E395E79093B2008093B1008091E4
:100E6000B1009091B2000F9708F459C08091B4007E
:100E7000843091F41092C4001092E2001092B900F4
:100E80001092C3009091BE0081E0282F291B20936F
:100E9000BE008093BF0041C080919E0090EB980FF0
:100EA000923088F49091B4009230B9F5803511F405
:100EB00081E501C082E58093B90081E08093BF00A5
:100EC00019BC18BC2AC08091CA00882331F18091D6
:100ED000BE00811122C08091B400833041F480E5CE
:100EE0008093B90081E08093BF0019BC18BC809149
:100EF000B400823091F480919E008F3F31F4809154
:100F0000E300882351F030DA08C086E98093C400FA
:100F10008091C4008093E200EED91092B4008091D9
:100F2000C8008230E8F18091CA008823E1F0809106
:100F3000E20084578B38A0F580919F009091A0002B
:100F400001969093A00080939F002091AF00309174
:100F5000B0002817390720F586E68093C4008093F7
:100F6000E20067D91DC08091B9008031C8F4E091DA
:100F7000B900F0E0E553FF4F80818F3F89F4809105
:100F80009F009091A00001969093A00080939F00F5
:100F90002091AF003091B0002817390708F401DB29
:100FA0008091CA00882391F08091C400823070F053
:100FB0008091C400863950F48091B1009091B200C4
:100FC0008C34910518F081E08093C100809160001D
:100FD00090916100009729F00197909361008093B0
:100FE00060008091600090916100892BD1F5909113
:100FF000B9008091CA00811104C081E0913041F4B0
:1010000008C09091E20081E0913019F09F3F09F013
:1010100080E02091AA0030E0811103C08EE190E0D1
:1010200002C08CE190E02817390734F480919D00CC
:101030008F5F80939D0004C010929D001092AC00C1
:1010400080919D00883068F081E08093AD008093AE
:10105000AC0010929D0088E391E090936100809332
:1010600060008091AC00882399F080919B00909162
:101070009C00019690939C0080939B00843F91403C
:1010800039F481E08093AB0010929C0010929B0099
:101090001092B6001092B50080919A008F5F8093F5
:1010A0009A00837019F486B1886486B9FF91EF9134
:1010B000BF91AF919F918F917F916F915F914F9170
:1010C0003F912F910F900FBE0F901F901895CF93C7
:1010D000DF931F92CDB7DEB717BA88E088BB85BB18
:1010E00083E087BB81EA8ABD81E083BF8CE087B95A
:1010F000A29A87EC86B9479A85B7877E806185BFBB
:10110000F8948BB78F7D8BBFA89584B7877F84BFFA
:1011100081B5886181BD11BCFAD81092A4001092EB
:10112000A3000091A3001091A4000038110508F05D
:101130000DC5C80143D5F82E8093EB00C801019678
:101140003DD5E82E8093C600C801029637D5D82E2B
:101150008093E700C801039631D58D3539F00C5FD7
:101160001F4F1093A4000093A300DBCF8F2D877037
:101170008093B9008F2D8695869586958F70809384
:10118000EA00FF1CFF24FF1CF092CA008E2D817024
:101190008093C900E1FA882780F98093ED008E2DB5
:1011A0008695869587708093EE00E294E69487E0BA
:1011B000E822E092C8008D2D81708093C500D1FA9D
:1011C000882780F98093E900D2FA882780F98093F4
:1011D000EC00D3FA882780F98093E000D4FA8827BE
:1011E00080F98093EF008D2D829586958370809392
:1011F000E3008091EC008093E5008AEF90E0DED47C
:101200009FEF980F9E3F10F48093620025D8E091E5
:10121000C800F0E0EE0FFF1FE45DFF4F8591949151
:101220009093B0008093AF008091C500882359F05F
:101230008091CA00811107C08091F100811105C021
:101240009CD9CAD902C01092B9008091B90081110D
:101250000CC08091CA00811104C08091C500811129
:1012600004C060E570E082E09ED81092F1008AEF41
:101270008093E60089E18093E800F894A89581B511
:10128000886181BD80E481BD7894912CA12C442497
:1012900043941FE0312E08E2802EBB24BA9488E3E9
:1012A000E82EFF24F3940CEF1AE095E0C92ED12C20
:1012B00055245A948091BD00811172C28091BE0064
:1012C000A816C1F0A090BE0019BC18BC8AEF90E02F
:1012D00099D76CE370E084E066D81092BF008091EB
:1012E000BE00882329F08091B9008093E60002C0F7
:1012F0005092E6009091B9008091E600981709F4A9
:1013000004C18091B900803140F52091B900822F4D
:1013100090E0FC01EB52FF4F30813093E100FC0183
:10132000E553FF4F80818093C7008091C700909163
:10133000E10099BD88BD211106C08091E500882398
:1013400011F081E004C08091E600811101C063D7F3
:101350008091B9008093E600D8C08091B900809355
:10136000E60019BC18BC8091B900803579F480E999
:1013700091E048D71092BF008091B900803509F004
:10138000C4C08091AA0060E55FD8F6CF8091B90013
:10139000813579F48AEF90E035D71092BF008091C3
:1013A000B900813509F0B1C08091A90061E54CD840
:1013B000F6CF8091B900823571F48AEF90E022D7A0
:1013C0001092BF008091B900823509F09EC062E59D
:1013D0008AE03AD8F7CF8091B9008B3549F48091F3
:1013E000B9008B3509F091C069E28EE0ABD7F7CF39
:1013F0008091B9008C3501F58091B9008C3509F0E8
:1014000084C0B8E07B2E8091B9008C3519F0A8E03B
:101410007A2E0DC068E284E195D77A947110F3CFEB
:10142000F6CF60E588E28ED77A94772029F3809111
:10143000B9008C35B1F3E0CF8091B9008D3549F515
:101440008091B9008D3511F5F4E07F2E8091B900BF
:101450008D3519F0EAE07E2E14C019BCB8BC85E0C9
:1014600090E0D0D6B9BC18BC81E490E0CBD67A9499
:101470007110ECCFEFCF88E490E0C4D67A94772057
:10148000F9F28091B9008D35B1F3DACF19BC18BCEF
:101490003CC08091B9008E35D1F48091B9008E3571
:1014A000A1F58CE291E0AED66DE78DE74BD76DE705
:1014B0008DE748D77FE0772E8091B9008E3569F7A8
:1014C00084E690E09FD67A947110F6CFE6CF8091B3
:1014D000B9008F35D1F48091B9008F35B1F48CE229
:1014E00091E090D660EF80EF2DD760EF80EF2AD7A4
:1014F00064E6762E8091B9008F3569F784E690E036
:1015000081D67A947110F6CFE6CF8091AD00882312
:1015100009F445C08091CA00882369F18091E200F6
:101520008823D1F1813011F08F3F61F487E08093FF
:10153000E20088E0AAD71092C4001092E200109254
:10154000C30012C083E0A1D78091E2008A3050F03E
:1015500090E0880F991F880F991FB6011CD36093E4
:10156000E20002C04092E2008091E200C4D68AEF1D
:1015700090E048D611C08091B900882369F080912D
:10158000B900813011F488E001C083E07ED78091FA
:10159000B900803108F405D81092AD0028C08091C0
:1015A000AB00882321F18091E9008823F1F080913C
:1015B000B900811104C08091E500811105C062E08D
:1015C00084EF91E094D711C080E025D684EF91E0BC
:1015D00019D681E020D684EF91E014D680E01BD6A6
:1015E00084EF91E00FD681E016D61092AB00809187
:1015F000C8008130B9F59091A900809162009817D8
:1016000088F18091A6009091A700892B59F58091CF
:10161000CA008823B1F08091E200823418F1282FAB
:1016200030E066E098D2A901481B5109CA01423452
:1016300051050CF481E48093E2008091E2005BD6D6
:1016400009C08091B900882369F08091B900803188
:1016500048F4A7D71093A7000093A60063E084EF97
:1016600091E045D78091AC00882329F044EE642EA8
:1016700047E5742E04C036E3632E7724739480917B
:10168000CA00811104C08091B900882349F080917B
:10169000CA00882309F45AC08091E200811156C023
:1016A00053D7892B09F052C08091B1009091B200BC
:1016B0006816790608F04AC08091AA008E3130F48D
:1016C0008091E500882311F080E0A5D581E090E0CD
:1016D00099D51092B2001092B1001092A70010920A
:1016E000A600F894A89584B7877F84BF81B58861E8
:1016F00081BD11BC789437981092B6001092B50055
:1017000023D7892B21F080E190E07CD5F9CF8BB7EE
:1017100080628BBF85B7806285BF85B7846885BFCF
:101720008B7F85BF889585B78F7D85BF8BB78F7D74
:101730008BBF8CE087B9A29A87EC86B9F894A895FC
:1017400081B5886181BD80E481BD78948091A500D8
:10175000882309F4AFCD1092A5008091E200882380
:1017600009F4A8CD82548D3B10F422E001C021E0A1
:101770008CE291E0298346D5298181E029834BD5EC
:101780008FEA90E03FD580E046D52981223029F4C8
:101790008FEA90E037D521E0F0CF2130E1F78ACD14
:1017A0008091BB00891571F09090BB008091BB00C7
:1017B000882341F084E189BD18BC84E690E022D5FD
:1017C00019BC18BC9091BD008091BC00981709F419
:1017D000A1C18091BD008093BC001092BA0080919D
:1017E000BD00873109F47CC0E0F48E3009F448C0B4
:1017F00028F4813059F1833091F1DFC08F3009F442
:101800005AC0853109F0D9C080E991E0FBD481E06C
:101810008AD68091BD008F5F8093BD001092BB007F
:1018200076C1883209F473C138F4883109F467C08D
:10183000893109F471C0C1C0843609F479C0853694
:1018400009F481C0893209F0B8C08CC080E991E008
:10185000D9D481E068D68091BD008F5F3AC1809174
:10186000BB00882359F08091BB00893038F4809107
:10187000BB00817084258093CA00AED682E037C158
:1018800046D5AAD68091EC008093E500E5D487E3A5
:101890008093620067E38AEF96D6E091C800F0E09B
:1018A000EE0FFF1FE45DFF4F859194919093B00080
:1018B0008093AF002AC11092BD0068E270E085E01D
:1018C00072D51092C4001092E2001092B90080917B
:1018D000CA00882309F41BC18091C4000CD517C12C
:1018E0008091BB00882351F28091BB0081708425D8
:1018F0008093EC008091EC008093E500BECF809156
:10190000BB00882339F08091BB00817084258093CF
:10191000E00062D683E0EBC08091BB00882309F42D
:10192000F4C08091BB00817084258093E900ECC0F5
:1019300068E270E083E037D519BCB8BCF092A7002C
:10194000E092A600E4C019BC18BC8091A60090915A
:10195000A700892B11F56091A900609362008AEFBE
:1019600032D61BC08091BB008823B9F08091BB00A8
:10197000873098F48091BB008F5F8093C8002CD68D
:10198000E091C800F0E0EE0FFF1FE45DFF4F85918E
:1019900094919093B0008093AF008091CA00882307
:1019A00021F084E0C0D585E003C088E0BCD589E0A3
:1019B0008093BD008093BC00AAC08091CA00882398
:1019C000C1F18091BD008530A1F0863079F184307D
:1019D00009F09DC08091BB00882309F49BCF8091C2
:1019E000BB00883008F096CF8091BB008093EE005A
:1019F0003CC08091BB00813019F41092C80013C024
:101A00008091BB00823009F460C08091BB008330BC
:101A100059F466C0882341F08091BB008170842511
:101A20008093EF0019D4D8D584E061C08091BB00C9
:101A300060C0E091BD008E2F90E0FC013497E7304C
:101A4000F10508F064C0E15FFF4F8091BB0009948D
:101A5000882309F45FCF8091BB008D3008F05ACF06
:101A60008091BB0081508093EA00F6D352CF882347
:101A700039F08091BB00817084258093C900ACD57A
:101A800085E035C0882339F08091BB0081708425C2
:101A90008093ED00A1D586E02AC0882351F0809183
:101AA000BB00883030F48091BB008093EE00D4D32B
:101AB00093D587E01CC0813021F41092C8008CD5EA
:101AC00015C08091BB00823039F44092C80084D5A3
:101AD00084E68093BD001BC08091BB00833031F44D
:101AE00068E270E060D48092BD0011C088E01BD530
:101AF0000EC0882351F08091BB00843030F4809177
:101B0000BB0081508093E30067D53092BD001092F6
:101B1000BB00D0CB8091BB00882321F08091BA001C
:101B20008E3770F48091BD00843609F4C3CB809168
:101B3000BB008111BFCB8091BA008C3D08F4BACBB9
:101B40008091BD008F5F8093BD00B4CB1092A40044
:101B50001092A3004ECB991B79E004C0991F9617F1
:101B600008F0961B881F7A95C9F780950895AA1BDF
:101B7000BB1B51E107C0AA1FBB1FA617B70710F078
:101B8000A61BB70B881F991F5A95A9F780959095AA
:101B9000BC01CD01089597FB072E16F4009406D0E2
:101BA00077FD08D0E4DF07FC05D03EF490958195E1
:101BB0009F4F0895709561957F4F0895E199FECFED
:101BC0009FBB8EBBE09A99278DB30895F894FFCF01
:101BD000380137059E009A0094008C008200760040
:101BE000680062005C005600500048009F009C00A6
:101BF0009700900087007C006F0065005F0059002F
:0A1C000053004C005B5C5D5E5F006A
:00000001FF
